:020000040000FA
:100000008A810C2A00000000A000030EA1000A084B
:100010008312A2000408A3008A11D8288B138B1B1B
:100020000E285E30A90060305A288B138B1B1528D0
:100030002630A90027305A288B138B1B1C2813301D
:10004000A90014305A288B138B1B23288930A90050
:100050000A305A288B138B1B2A28D130A900043070
:100060005A288B138B1B3128E830A90002305A28FC
:100070008B138B1B3828F430A90001305A288B13BE
:100080008B1B3F284930A90001305A288B138B1B4A
:1000900046283130A90001305A288B138B1B4D287C
:1000A0002730A90001305A288B138B1B54280530A8
:1000B000A9000130AA002B148B172B185C2808000C
:1000C0008B138B1B6028BC30AC00BF30A5288B1372
:1000D0008B1B67285E30AC006030A5288B138B1B10
:1000E0006E282630AC002730A5288B138B1B752873
:1000F0001330AC001430A5288B138B1B7C2889305F
:10010000AC000A30A5288B138B1B8328A130AC00D0
:100110000830A5288B138B1B8A28D130AC00043003
:10012000A5288B138B1B9128E830AC000230A52842
:100130008B138B1B98283130AC000130A5288B1312
:100140008B1B9F280530AC000130AD00AB148B1722
:1001500008008E018F01C528DF308E00BF30C42813
:1001600000308E00C030C42814308E00FE30C42809
:10017000B8308E00FE30C428FA308E00FE30C4281D
:10018000DF308E00FF30C4288F008B138B1BC528F7
:10019000101463000C1CC92810100C108B170800D9
:1001A00000308A0024038207E9341634FF34FF3418
:1001B0008B1EF7290B1DF7290B110E08E8070F08F6
:1001C000E8072B1CE828A90BE828AA0BE8282B1025
:1001D000AB1CEF28AC0BEF28AD0BEF28AB10071BC7
:1001E0004B292F180129CC0B4B29CD0B4B29AF14D0
:1001F000871B0529AF103130CC000130CD002F1402
:100200004B29CC0B4729CD0B4729060EFC00FC0CD3
:100210000730FC05AF1822290D2901308A00031090
:100220007C0D820725143629A51436292515362973
:10023000A515362925163629A51636292517362956
:10024000A517362901308A0003107C0D820725107E
:100250003629A510362925113629A511362925124A
:100260003629A512362925133629A5132F100A3051
:10027000CC000130CD000615861420308607060715
:10028000031C46291F308605061586104B29871F3B
:100290004B29AF1405292F1DA529AF1D5C29CE0BB5
:1002A000A529CF0BA5295008400203195929AF11E0
:1002B0009529AF112F11A529003040020319A52956
:1002C00010305002031D8529103040020319702997
:1002D00010304002031C6E29851579298511792972
:1002E000121197010711D130CE000430CF00AF15A5
:1002F000A5291708031DA5299101503095000C3040
:1003000097001215D301D401A52948305002031DCE
:100310009529483040020319702948304002031CD7
:10032000932985157929851179292C305002031DCF
:10033000A5292C304002031970292C304002031CDF
:10034000A32985157929851179292F1ED7294008D8
:1003500051020318B229400852020318C0295C1543
:100360008515BE2904305D02031DBD295C1DBD2914
:100370002F12121197010711D7298511AF13AF1250
:10038000AF1BD7292F1FCE29861DCD29D70BD729E3
:10039000D80BD729AF172F13D7292F13861DD7298D
:1003A0002F17F430D7000130D8004008DB0020249C
:1003B0005C1EE62905092739E4000319F7295C12B8
:1003C000DC16D130E2000430E300F729DC1EF72907
:1003D000050927396402031DF429E20BF729E30B11
:1003E000F7296408E5005C17DC125C16F7298B1806
:1003F0008B1083168C1D002A83128C1D002AD82591
:100400008312022A83122308840022088A00210E04
:100410008300A00E200E090020308300C13081002F
:100420008E018C018D0137308500093086009930AE
:10043000870000309800FF3099005E3093007C30D8
:100440009200831240308B008C018D0108308500B2
:10045000E030860078308700980107309000013046
:100460009200910136309400203084008001840A8B
:1004700080300402031D362AA03084008001840FDE
:100480003E2A8C118312141394138C1D422A8C1152
:100490001308141B422A83161419422A8312AA270E
:1004A0004C3C031D422AAA27FF00163C031D422A8A
:1004B000AA27FF077F3C031D422AAA277F07013E88
:1004C000031D422AAA27141B422A8316141D422AFE
:1004D00083127F085E3E930014168C1D6D2A8C11CA
:1004E0000230D6000030D5001030D1004830D200A4
:1004F000B030CA0083168C15831281010B118B1644
:100500008B17A026AB198F2A8B138B1B842AAB1F4A
:100510008F2A2B1A8E2AAB1EAB158F2AAB138B1387
:100520008B1B8F2A2B1FA82A10304002031DA22AE2
:1005300085119101503095000C3097001215D301B0
:10054000D401A82A00301702031DA82AAB15A82A37
:100550008B17DC1DAD2ACB01AF2A5C1CC62A0717FE
:1005600087124B08031DC22A8B138B1BB42A12114E
:10057000970107118B100B1663008B100B128B1752
:10058000061CAF2A5C10DC108716812ADC18AF2A03
:10059000671CD12AAB1BD12A67105D080F39A80050
:1005A000D222812A02308A0028088207E62AE72A16
:1005B000E72AEB2A112B112B1A2BE72AE62AE62A27
:1005C000E62AE62AE62AE62AE62AE62A08002C3067
:1005D000D0002F1508002630D1003230D200503024
:1005E000D5000430D6002F162F11AF11AF13AF1264
:1005F0005C114008DB001708031D062B91015030E9
:1006000095000C3097001215D301D401E030860418
:100610000615861007130130CC000130CD002F14D1
:1006200008001030D1004830D2000030D50005302D
:10063000D60008002C30D0002F1508001030FF0025
:10064000B001B101B201B3018323031C812B260841
:10065000B007031C2C2BB10AA61F2F2BB1032708B0
:10066000B207031C342BB30AA71F372BB303FF0BAE
:10067000242B0430FF00B10CB00CB30CB20CFF0BF8
:100680003B2B3008A6003208A7000C30A800303001
:100690008400D42326028000000D031C512B800906
:1006A000800AE5232702FE007E0D031C592BFE095C
:1006B000FE0A7E088007840AA80B492B0C30FF0035
:1006C00030308400FF30FE0000087E02031C6A2BDD
:1006D0000008FE00840AFF0B642B30308400000801
:1006E0007E020319752B840A6F2B303084020408B4
:1006F000A800002486000408A80010248700031422
:10070000822B031008008B138B1B832B7A309200F3
:1007100091013A3083169200831212158C10051C39
:10072000972B8C1C8F2B031012118B1708001211A2
:100730009101263083169200831212158C10051831
:10074000A42B8C1C9F2B932B0508B400B501003003
:100750009200910126308316920083123710B71051
:1007600012158C108C1CB22B8C10B50FB82B932B40
:100770000508B60034063605B400B41CC82B37187B
:10078000932B3508A6003714B71CC82B0314942BE1
:10079000341DD12BB718932B3508A700B714371881
:1007A000C62B3608B400B22B03308A002808820713
:1007B00000344A34403425340034DB34C034B63499
:1007C000BF34DB3400342534413403308A00280838
:1007D0008207003425340034DB34BF34B634C034EF
:1007E000DB340034253440344A3441340000000006
:1007F00000000000000000000000000000000000F9
:1008000004308A0028088207FE34FD34FB34F734B4
:10081000EF34DF34BF347F34FF34FF34FF34FF3430
:1008200004308A0028088207FF34FF34FF34FF3485
:10083000FF34FF34FF34FF34EF34DF34BF347F3410
:10084000D30F2E2CD40A5408083903192E2CD301A7
:10085000D4017D30150203182E2C950AAB1D372DBF
:10086000411C472C051E3E2CC70A05304702031DBC
:100870003F2CC701C401C501C601C02DC701C40A70
:100880000A304402031DC02D4110C114C02DC11CEB
:10089000562C051A4E2CC201C301C02DC20A0A30C3
:1008A0004202031DC02DC1104115C02D411D6C2CED
:1008B000D301D401051E642CC401C501C601C20FB9
:1008C000C02DC30FC02DC12DC40A0A304402031D20
:1008D000C02D4111C115C02DC11DD22CD301D40191
:1008E000051A7A2CC701C40FC02DC50FC02DC60F25
:1008F000C02DC12DC70A0A304702031DC02D420872
:10090000FC004308FB00FA010310430C420CFC07F7
:100910000318FB0A0310430CFB070318FA0AC82547
:10092000031CC52C4208FC004308FB00FA0103101D
:10093000FC0DFB0DFA0D4208FC070318FB0A4308E7
:10094000FB070318FA0AC825031CCE2C4208FC003A
:100950004308FB00FA010310FC0DFB0DFA0DFC0D22
:10096000FB0DFA0D4208FC070318FB0A4308FB07BE
:100970000318FA0AC8250318C52C8511C11141179F
:10098000C701C401C501C601C02D4708C200C3018B
:10099000C401C501C601C1114115C02DC1114116C7
:1009A0008511C02D411EE42C051AE02CC40FC02D6A
:1009B000C50A03304502031DC02D4112C116C02DCA
:1009C000C401C501C601C02DC11EFF2C051EFD2C92
:1009D000C70A0A304702031DC02DC1011030C000F4
:1009E000121197010711AB112B16C401C501C601E5
:1009F000C201C301C7018515C02DC701C02D411F0C
:100A00000F2D051A0B2DC40A0A304402031DC02DF8
:100A10004113C117C02DC401C501C601C02DC11F9E
:100A2000262D051E1F2DC70A0A304702031DC02DA3
:100A300002304502031C262DC1134117C02DC40FDF
:100A4000C02DC50FC02DC60FC02DC12D4114C4012E
:100A5000C501C601C201C301C7018515910150300E
:100A600095000C3097001215D301D401C02D2B1E18
:100A70007B2D400C0318782D051A742DC40A0A30FA
:100A80004402031DC02D8519512DC00A400C0318C6
:100A90004C2D8A15E3218A1148304002031DC02DD8
:100AA0006E2DC003400C0318582D8A15E3218A11BE
:100AB0001030400203196E2D103040020318C02D73
:100AC0002B12AB160330C000851191014D309500FB
:100AD0002C3097001215D301D401C02D2F1AC02D30
:100AE000121197010711C02DC401C501C601C02D07
:100AF000051E742D3E2DAB1EC02D01304002031D7E
:100B0000952D051E892DC70A0A304702031DC02DE9
:100B1000ED2CC701C40FC02DC50A02304502031DCC
:100B2000C02D0330C0008511C02D02304002031DCE
:100B3000B02D051EA42DC70A0A304702031DC02D83
:100B40008511AB122B167B2DC701C40FC02DC50A12
:100B500002304502031DC02D0430C0008515C02D94
:100B600003304002031DB82D051A832DC701C02D87
:100B700004304002031DBF2D051A9B2DB62DC12D3B
:100B80000800C101C001AB15121197010711C02D5A
:100B90004408FC020318D02DFF30FB07031CFA03A6
:100BA0004508FB02031CFA034608FA027A0D080006
:100BB0001308FC00141B932E8C11831614199B2E02
:100BC000941AE42D8312962E8312671DEE2D4C305D
:100BD0007C02031D932E6711E715922EE719052E4F
:100BE000671EF72D6712E7167C08EB00922EE71EB2
:100BF000932EE71249086B07FB007C07013E031D9B
:100C0000932E7B085E3EC8007C2EFC1F0C2EE71145
:100C100067167C08C900922E20307C02031D132E1B
:100C20002508C800922E21307C02031D1A2E400890
:100C3000C800922E22307C02031D2C2E2F1E172E50
:100C4000AF1F172EAF1A172EFD308519282E003032
:100C50005B078038C800922E23307C02031D362E9D
:100C6000C80117080319922EC80A922E24307C025C
:100C7000031D5D2E5C1F5B2E6508FC00FC0C7C0CCC
:100C8000083965040F39A8004726C800922E06309F
:100C90008A00280882078734813487348334873474
:100CA000873480348334823487348734873484347F
:100CB000873484348734C801922E25307C02031D8A
:100CC000652EC8016718C80A922E27307C02031DC2
:100CD0006B2E6908702E28307C02031D732E6A0863
:100CE000C800E710922E26307C02031D7B2EC8011F
:100CF000E718C80A922E922E20304B020319922E2A
:100D00004B084A078400D0300402031C892EE030CF
:100D1000840749088000840A6B088000CB0ACB0A4C
:100D2000922E831208001413941314166715E711FA
:100D30006712E712922E8312480893001416922E1F
:100D40008B138B1BA02E4B080319A82F4A08840075
:100D5000F0300002031DB42E840A000C0318B22EDA
:100D60002B139E2F2B179E2F000D031C9E2F000868
:100D70001F39A80016302802031CBF2E9E2F0630F4
:100D80008A0028088207332F352F482F502F6A2FCB
:100D9000752F792F7D2F9A2FDE2ED92ED82ED82E73
:100DA000D82ED82ED82ED82ED82ED82EFA2EE22EE7
:100DB0009E2F840A0008A8008A154A29AF13AF1293
:100DC0002F139E2F840A2F122F11AF11AF13AF12C2
:100DD0005C114008DB0000080319F72E0130000207
:100DE0000319F42EDC159E2FDC145C109E2F5C146E
:100DF000DC109E2F840A5D08E600000203199E2F76
:100E00000008DD005C12DC12AF13AF122F122F119D
:100E100009305D0203192E2F0C305D0203192C2FAF
:100E2000671401305D02031D1D2F0A30660203198D
:100E3000322F023066020319322F0030C0000A3010
:100E40005D0203192C2F02305D0203192C2FAB1702
:100E50002B12AB12C1019E2F8001E32E2F12121113
:100E6000970107119E2FAF169E2F840A00080319C1
:100E7000442FE03086040615861007130130CC009D
:100E80000130CD002F149E2F0717061186109E2FBC
:100E9000840A000EF039D500000E0F39D6009E2FBF
:100EA0002B1EA82FAF13AF122F12840A0008031DA8
:100EB0005D2F1030D0002F159E2F01300002031D32
:100EC000632F2C305A2F02300002031D692F483047
:100ED0005A2F9E2FAB199E2FAF13AF122F122F1127
:100EE000AB172B12AB12C1019E2F840A0008D10050
:100EF0009E2F840A0008D2009E2F840A000803193E
:100F0000952F2F162F11AF11AF13AF125C114008A0
:100F1000DB001708031D9E2F9101503095000C3007
:100F200097001215D301D4019E2F2F121211970191
:100F300007119E2F5C13DC125C169E2FCA0ACA0A88
:100F4000D0304A02031CA62FB030CA00CB03CB031B
:100F50008B1708008C1DAA2F8C11130808000000A5
:100F60000000000000000000000000000000000081
:100F70000000000000000000000000000000000071
:100F80000000000000000000000000000000000061
:100F90000000000000000000000000000000000051
:100FA0000000000000000000000000000000000041
:100FB0000000000000000000000000000000000031
:100FC0000000000000000000000000000000000021
:100FD0000000000000000000000000000000000011
:100FE0000000000000000000000000000000000001
:100FF00000000000000000000000000000000000F1
:1010000008308A00280882070A340034103400347B
:10101000133400341834003450340234543402345D
:101020005C3402346334023466340234693402348A
:101030006C3402346F340234723402347B34023440
:10104000813402343934023405340334DF34023459
:1010500009340334D134023402340334F234023418
:10106000EB340234FE340234EF340234DB34023425
:10107000F5340234F9340234CE3402342B340234E1
:101080005734003488340034B0340134D03401345F
:10109000513400348234003432340034B0340034FB
:1010A0007D34003402340234E7340134BB3401347B
:1010B000B634013415340234F83401341E340134AA
:1010C000283401342C3401343334013438340134BD
:1010D000423401347D340034DC340134D7340134FB
:1010E000F3340134A9340134EB340134CB3401340A
:1010F000C03401343034023406340234493402340A
:101100003F3402344D340234283402343334023450
:10111000123402340A34023442340234D4340034F7
:101120004C340434A6340134A3340134463401343D
:101130004B3401344E340134553401345C340134C1
:101140006034013465340134693401346E3401345F
:10115000743401347B3401348234013489340134F1
:10116000933401340D34033412340334183403340B
:101170001E34033423340334353403343A34033413
:1011800029340334A7340334AD340334B234033484
:10119000B5340334BD340334C3340334C8340334A6
:1011A000CD340334D2340334D7340334DC34013443
:1011B00033340134EB3402347B340234C034013430
:1011C00049340234063401340D340134103401340E
:1011D000183401349D340334A3340334E834003428
:1011E000E134033442340434000000000000000005
:1011F00000000000000000000000000000000000EF
:1012000009308A002808820735340334B6340034A4
:10121000BC340034C8340034CC340034DB34003403
:10122000ED340034F2340034F8340034E63403345E
:10123000F0340334863402349E3402348C34023465
:101240004934043493340234963402349A340234E8
:101250000034003404340034BA340234A334023489
:101260004234013433340134D0340134B0340134E5
:101270008834003457340034DB340034FF0068080D
:101280000107FE007F0803194929FE0203184529BA
:101290007E07080009308A002808820771297F2903
:1012A00087298B298F299129932997299B299F2960
:1012B000A129A529A929AD29B929BD29BF29C12954
:1012C000C329C529C729C929CB29CD29CF29D12986
:1012D000D329D529D729D929DB29DD29DF29832954
:1012E000E12904303E21003EA8000310A80D002093
:1012F000E900A80A0020EA00E7148A119E2F0C30AA
:101300003E21043E74290E303E21103E74290F30D8
:101310003E211E3E742918303E212D3E7429453051
:1013200074294630742902303E21473E74290E301C
:101330003E21493E742907303E21573E74295E30D4
:10134000742910303E215F3E742904303E216F3EE7
:10135000742905303E21733E74290030A800031023
:10136000A80D0021E900A80A0021EA00E7148A116B
:101370009E2F09303E21013EAE290A30AE290B30A6
:10138000AE290C30AE290D30AE290E30AE290F300B
:10139000AE291030AE291130AE291230AE291330EB
:1013A000AE291430AE291530AE291630AE291730CB
:1013B000AE291830AE291930AE291A30AE291B30AB
:1013C000AE291C30AE295508D3020318E929FF3095
:1013D000D4075608D4020319112A0318022A150843
:1013E000031DF629170E03390319112A170E0339A5
:1013F000FF3E031CFE29F0309707112A3C3097006E
:101400009503112A7D3015020318112A170E013E8B
:10141000033903190E2A10309707112A0C30970050
:10142000950AD301D401080000000000000000006C
:1014300000000000000000000000000000000000AC
:10144000000000000000000000000000000000009C
:10145000000000000000000000000000000000008C
:10146000000000000000000000000000000000007C
:08400000813F813F803F823FB8
:00000001FF
